:020000040800F2
:10000000901C00202901000831010008330100087C
:100010003501000837010008390100080000000020
:100020000000000000000000000000003B0100088C
:100030003D010008000000003F01000849250008BC
:100040004301000865160008430100084301000849
:100050004301000843010008E505000851060008B7
:100060007106000891060008B1060008790300082F
:100070004301000843010008430100084301000850
:100080004301000843010008430100084301000840
:100090004301000843010008D1060008430100089D
:1000A00043010008430100084301000869270008D4
:1000B000B92700080D280008430100084301000883
:1000C000F5110008811100084301000843010008F0
:1000D0004301000843010008430100080506000829
:1000E00043010008430100084301000843010008E0
:1000F0004301000843010008430100085528000897
:100100009D2800084301000843010008430100083E
:1001100043010008DFF80CD000F07EF800480047EB
:10012000E1330008901C002006488047064800473D
:10013000FEE7FEE7FEE7FEE7FEE7FEE7FEE7FEE797
:10014000FEE7FEE7B92600081501000840EA0103B2
:100150009B0703D009E008C9121F08C0042AFAD27D
:1001600003E011F8013B00F8013B521EF9D2704741
:10017000D2B201E000F8012B491EFBD270470022E9
:10018000F6E710B513460A4604461946FFF7F0FF96
:10019000204610BD2DE9F05F0546002092469B46A3
:1001A00088460646814640241BE02846414647468D
:1001B000224600F020F853465A46C01A914110D307
:1001C00011461846224600F039F82D1A67EB01084F
:1001D0004F4622460120002100F030F817EB0009BD
:1001E0004E41201EA4F10104DFDC484631462A4678
:1001F0004346BDE8F09F202A04DB203A21FA02F0B2
:100200000021704721FA02F3D040C2F12002914050
:100210000843194670470000064C074D06E0E068A9
:1002200040F0010394E8070098471034AC42F6D33D
:10023000FFF774FFAC3C0008CC3C0008202A04DB2C
:10024000203A00FA02F1002070479140C2F12003E9
:1002500020FA03F31943904070470000F0B5274A95
:100260008CB0802420270021A2F5A5656E4601EB05
:10027000C103C3EB811305EB430303F0704CC3F3DD
:1002800013030CEB43131B1B03F100733C3346F8C1
:100290002130491C89B20C29E9D300232AE019072F
:1002A00009D156F8214004EB870446F82140491C47
:1002B00089B20C29F5D30021DFF844C0118056F82B
:1002C0002140DCF8105024886D5CAC401588491C36
:1002D0002C4389B214800C29F1D30021921C56F8CA
:1002E0002140241F46F82140491C89B20C29F6D32D
:1002F0005B1C9BB28342D2D30CB0F0BDA40F002094
:10030000140A00202DE9F04186B04FF4007001F08E
:1003100093FB4FF4806001F08FFB684600F0E9FC2E
:100320000125AF03124ECDE9007500246946304621
:10033000039400F09FFC3946304600F0C5FCEE0304
:10034000DFF83080CDE9006569464046039400F04F
:1003500091FC3146404600F0B5FCCDE901456946C7
:1003600040460097039400F085FC06B0BDE8F0819C
:1003700000400240003C02400B4810B5016889076C
:1003800011D5416841F00201416008480121017026
:10039000002141800448083000F00CF8BDE810400E
:1003A000034801F058BC10BD000002404A00002084
:1003B000003C0140016821F00101016070470161CA
:1003C0007047026822F02002026002680A4302605D
:1003D0007047026822F01002026002680A4302605D
:1003E000704710B5044608680B46A0604868E06096
:1003F00089682046FFF7EDFFD868606020461969DC
:1004000000F032F82046596900F01EF8204699693C
:1004100000F032F82046D96900F01EF82046196A2B
:10042000FFF7CFFF2046596A00F02EF82046996A60
:10043000BDE81040AFF30080026822F48042026001
:1004400002680A4302607047026822F0800202607C
:1004500002680A4302607047026822F44062026048
:1004600002680A4302607047026822F0400202609C
:1004700002680A4302607047026822F44072026018
:1004800002680A4302607047026822F44052026028
:1004900002680A4302607047016821F001010160AF
:1004A0000021016041608160C1602149204A083912
:1004B000904203D1486840F00F0006E01C4A143215
:1004C000904204D1486840F0F00048607047184AF4
:1004D0002832904203D1486840F47060F5E7144A2E
:1004E0003C32904203D1486840F47040EDE7104A36
:1004F0005032904203D1486840F47020E5E70C4A3E
:100500006432904203D1486840F47000DDE7084A45
:100510007832904203D1486840F07060D5E7044AD1
:100520008C329042D2D1486840F07040CDE7000054
:10053000080002400021016041608160C1600161EA
:1005400041618161C1610162416281627047000065
:1005500070B50F4C0026268060800E48A060207C7D
:1005600040F0010020744FF08045AE84286840F0D0
:100570000100286019B1208861888842FBD300F00F
:100580000BF8286820F001002860267470BD000078
:10059000F0090020A40F002003480168034A928A52
:1005A000114301607047000014340240140A002017
:1005B000094900220A80488008488860087C40F089
:1005C000010008740648028005482438016841F09B
:1005D0000101016070470000F0090020841600202E
:1005E0002404004006480168C90708D004491439AA
:1005F0000968C90703D00121016001F0C5BC70473B
:10060000140401400E4810B50068800417D50C484A
:1006100014380068800412D50A48816821F001016D
:1006200081600948018821F040010180401400F0F8
:100630005FF806488088BDE8104001F0A9BB10BDF6
:100640001404014000000240003C0140140A002054
:1006500006480168890708D50449143909688907DB
:1006600003D50221016001F08FBC704714040140E2
:1006700006480168490708D504491439096849073B
:1006800003D50421016001F07FBC704714040140D0
:1006900006480168090708D504491439096809079B
:1006A00003D50821016001F06FBC704714040140BC
:1006B00006480168C90608D5044914390968C906FD
:1006C00003D51021016001F05FBC704714040140A4
:1006D00006480168C90508D5044914390968C905DF
:1006E00003D58115016001F04FBC7047140401402F
:1006F0000149086070470000140401400649096878
:10070000014206D0044914390968014201D0012090
:10071000704700207047000014040140034B00297B
:1007200003D199180A6882430A60704700040140A7
:1007300010B504460179006800F02EF86179206850
:1007400000F00EF82279A1792068BDE81040FFF78B
:10075000E5BF0021016001710C2242718171704777
:1007600030B50C4B0B4D08331A6882431A601A1DC2
:10077000146884431460102904D029440A68024391
:100780000A6030BD196801431960116801431160A6
:1007900030BD000000040140064A10B513688343D1
:1007A0001360131D1C6884431C6011440A680243D3
:1007B0000A6010BD0004014009480168094BD8884F
:1007C00001400948428C0A404284084909691A8953
:1007D0001140828C0A408284816A491C8162704780
:1007E00010380240140A00201C060020004002407D
:1007F00070B500F031F8174D044602280ED04FF0C6
:10080000020116D128896A8800EB01039A4208D9AF
:10081000501A80B2688000F015F918E04FF004011A
:10082000EFE7688000F00EF90120A875288B401CC6
:100830000CE0012C0BD168880144E888814200D289
:1008400088B2688000F0FEF80020A8752883204652
:1008500070BD00001C06002070B5334D688C334E0F
:10086000F1880840A8816889E881A88C318908400E
:100870006882288AA882E87D002138B1012802D048
:100880000024204670BD02242983FAE7A889EA895A
:100890001040EA89904205D1688AAA8A1040AA8A43
:1008A00090422AD0A87D012825D1E87E012822D1B6
:1008B000288BFA281FD3298395F82100D8B9002165
:1008C0000122EB8902FA01F0034206D0AB89034210
:1008D00003D16B8983436B816B89AB8A034206D05A
:1008E0006B8A034203D12B8A83432B82288A491CBB
:1008F000C9B21029E5D30224C3E7688908B9288A58
:1009000008B10124BDE70224642002F036FD1F2156
:100910000022602001F0DEFC642002F02EFDF08851
:10092000688130892882ACE71C060020140A002068
:1009300000B587B0802001F07FF8684600F0D9F953
:1009400010200090002003900220019009200590C3
:100950006946024800F08EF907B000BD003402403D
:1009600070B5354C6078012505285ED2DFE800F0CF
:10097000030E283E5300E07D022856D0607F401CC5
:100980006077607F88B36570A5764EE0E07D60BBE0
:10099000A06A032849D9FFF72BFF0221022802D0C1
:1009A000012804D041E0A07D012803D03DE0A07FD4
:1009B000032801D3617038E0A07F401CA07734E0A9
:1009C000642002F0DAFC1D4800250178032902D2D8
:1009D00000F0C6F808E005700320607044F2FF30B4
:1009E00060844FF40040A084A5621EE0E07D10B951
:1009F000A06A032802D8E07D012801D1FFF7F8FEA4
:100A0000E07FA12803D3E576042060700DE0E07F4D
:100A1000401CE07709E0E07D10B9A06A032802D805
:100A2000E07D012801D1FFF7E3FE0548C18861841C
:100A30000089A08470BD00001C0600204800002032
:100A4000140A00200146014801F0FBBF00340140B8
:100A50000449012008700448016841F00101016067
:100A6000704700001C060020001000401FB504461F
:100A7000102000F0F1FF684601F0B4FF3F20641E33
:100A8000ADF80000ADF8044000200C4CADF80600B5
:100A9000ADF802006946204601F04AFF01212046D8
:100AA00001F0D5FF0121204601F0D5FF204601F0DD
:100AB0000BFF204601F0D2FF1FBD000000100040D8
:100AC0007FB50D462349B1FBF0F04FF47A71B0FBCE
:100AD000F1F44FF4005000F0D1FFFFF729FF684612
:100AE00001F080FF641E40F2E730ADF80040ADF841
:100AF00004000024184EADF80640ADF802406946E7
:100B0000304601F015FF154AB0151146908170204E
:100B10001080D48108205081022010810420908010
:100B200001205080D580304601F0A2FF304601F010
:100B3000CBFE09481030016821F001010160304608
:100B400001F091FF304601F0E9FF04482C38458060
:100B50007FBD00000020A1070034014048060020AE
:100B600070B5184D044603202978B1FBF0F200FB64
:100B7000121262B1B1FBF0F200FB1212012A09D08D
:100B8000B1FBF0F200FB121002280AD00EE001F0D7
:100B900087FC08E048F240410022462001F09AFB21
:100BA00001E001F0EEFB052002F0E7FB2878401C95
:100BB000C0B22870032804D1002028702078401C7F
:100BC000207070BDE800002010B514074FEA427293
:100BD0004FEAD2624FF00F0303FA02F301FA02F177
:100BE00004D5426A9A431143416210BD026A9A4396
:100BF0001143016210BD10B5C36A52000324944032
:100C0000A34391401943C16210BD0000084A20F07F
:100C1000030310B51A4453688007C00E3F24844074
:100C2000A3435360536881400B43536010BD0000E1
:100C300000000140006980B2704770B5056853003C
:100C400003269E4001F00304B5439C402C430460FE
:100C5000012905D0112903D0022901D0122908D178
:100C6000436801249440C1F30011A3439140194308
:100C7000416070BD70B50C46064600251DE00120A0
:100C8000A840014218D02A4630466169FFF79CFF10
:100C90002A4630466168FFF7D0FF2A463046A168F1
:100CA00000F014F82A463046E16800F019F82A46A8
:100CB00030462169FFF79FFF6D1C216831FA05F06E
:100CC000DDD170BD816270478161704710B5C36826
:100CD000520003249440A34391401943C16010BDC6
:100CE00010B5836801249440A34391401943816067
:100CF00010BD4FF6FF7101600021C16041600F22FD
:100D00008160C0E904127047F8B505460024C0E0D0
:100D100014B962A002F09EF880261CB9314664A086
:100D200002F098F800223146412001F0D3FA642005
:100D300002F023FB00261CB9314661A002F08AF8BC
:100D400000223146422001F0C5FA642002F015FB72
:100D500007261CB931465EA002F07CF8002231461D
:100D6000472001F0B7FA642002F007FB48F634266A
:100D70001CB931465AA002F06DF8002231464820D5
:100D800001F0A8FA642002F0F8FA4FF404461CB906
:100D9000314657A002F05EF800223146492001F0AA
:100DA00099FA642002F0E9FA19261CB9314654A0D8
:100DB00002F050F8002231464A2001F08BFA6420FC
:100DC00002F0DBFA00261CB9314651A002F042F8CD
:100DD000002231464B2001F07DFA642002F0CDFA6A
:100DE00042F208061CB931464DA002F033F8002249
:100DF00031464C2001F06EFA642002F0BEFA49F64A
:100E000001661CB931464AA002F024F8002231469E
:100E10004E2001F05FFA642002F0AFFA4FF4C046B2
:100E20001CB9314646A002F015F8002231464F2089
:100E300001F050FA642002F0A0FA454800F060F991
:100E4000444B454E002404EBC40204EB4400C2EBC7
:100E50008412002103EB800006EB420230F811708F
:100E600002EB410C491CC9B2ACF80C700629F5D351
:100E7000641CE4B20C2CE6D3384801221146837A74
:100E80004020009301F03CFA642002F076FA641CE2
:100E9000E4B2AC42FFF43CAFF8BD00000A0A726550
:100EA00067697374657220636F6E6669670A000014
:100EB0007265675F34313A307825780A00000000A7
:100EC0007265675F34323A307825780A0000000096
:100ED0007265675F34373A307825780A0000000081
:100EE0007265675F34383A307825780A0000000070
:100EF0007265675F34393A307825780A000000005F
:100F00007265675F34413A307825780A0000000046
:100F10007265675F34423A307825780A0000000035
:100F20007265675F34633A307825780A0000000004
:100F30007265675F34653A307825780A00000000F2
:100F40007265675F34463A307825780A0000000001
:100F5000EA000020500000207C0A0020140A002033
:100F60002DE9F0470024642002F0EFF9642002F03C
:100F7000ECF9642002F0E9F94D4D00224FF64003F0
:100F8000A87A401E81B2104602F094FA4FF48046CF
:100F900001F086FA642002F0F0F901F087FA64208B
:100FA00002F0EBF9022C05D100223346114610461F
:100FB00002F08AFA00210A46442001F08BF96420ED
:100FC00002F0DBF9641CA4B2032CE1D3DFF8E49057
:100FD000DFF8E4A000244FF6FF7800231A461946F4
:100FE000184602F071FAA97A012001F04FF9A87AA7
:100FF000401DC0EB001000EB800108EA810002F008
:10100000BCF94846FFF716FE07465046FFF712FEAA
:1010100027F43C4100F4004001430CD0032C17D2CC
:101020002648468101F042FA4FF4FA7002F0A5F921
:10103000022C07D00CE000231A461946184602F08D
:1010400043FA09E000231A461946184602F03CFA12
:10105000641CA4B2032CC0D30320FFF755FE002468
:1010600048F6424635461CB9314615A001F0F2FE5D
:1010700000222946462001F02DF9642002F07DF976
:101080003F251CB9294612A001F0E4FE00222946A2
:10109000602001F01FF9642002F06FF9641CA4B213
:1010A000032CDFD3BDE8F0470DA001F0D3BE000054
:1010B000140A00200038024000400240841800203A
:1010C0007265675F34363A307825780A0000000090
:1010D0007265675F36303A307825780A0000000084
:1010E0006261636B6C6967687420647269766572AB
:1010F00020696320696E697420646F6E650A000060
:101100002DE9F84FDFF870A081460022194B1B4FE4
:101110009AF800609AF801C01BE0002115E033F84E
:10112000020B39F8124000F00F05C0F30618C00A90
:1011300005EBC80500EBC008C8EB801007EB4000CA
:1011400000EB4500491C8481C9B28E42E7D8521C8D
:10115000D2B29445E1D8BAF80C0000909AF80A305F
:1011600008220121502001F0CBF8BDE8F84F64209F
:1011700002F003B9DC340008140A00207C0A0020C5
:1011800010B5194C204600F08CF9B0F5806F06D0F0
:101190001649C20509D5088820F480700AE0204667
:1011A000BDE81040124900F04EB9820504D5088808
:1011B00020F40070088010BD020503D5088820F4D3
:1011C0000060F7E7C20403D5088820F48050F1E7F7
:1011D000420403D5088820F48040EBE70004EAD5F8
:1011E000088820F40040E5E700580040145800400B
:1011F000000400102DE9F047DFF840A1504600F050
:1012000050F9C1033ED4DFF838814C4A4D4F4E4B64
:1012100001251032DFF834917C1FA0EB08014FF05C
:10122000000CA3F58076404552D013DCB0F1021FCC
:1012300026D003DC48B110281ED179E04038B0F543
:1012400000306FD04249C84216D15046BDE8F04741
:1012500000F02EB9DFF8FC80A1EB080041450FD06B
:1012600004DC022910D0042906D131E03E2859D0EF
:101270007E38B0F5802F07D0BDE8F04700F0A4B964
:10128000A4F80AC0BDE8F087A4F80CC03078202884
:101290000FD1707801280CD1B078012802D0022833
:1012A00004D006E0F078202821D002E0F078202851
:1012B0000CD0484650F8061F196041685960B9F8CB
:1012C0000E00188118781080A581DBE73878FAE7DE
:1012D0003078202811D1707801280ED1B0780128FB
:1012E00002D0022806D008E0F078202805D1A078A6
:1012F0001080C7E7F078202810D0484650F8061F25
:10130000196041685960B9F80E001881207B00F01F
:101310000F00195C1180401CA081B3E7A089395CE3
:10132000F8E7FFE7A07A11883154401C6081A9E7F3
:10133000504600F0BDF82581A4E7000000580040A9
:101340008000060029000020140200205C380008FC
:101350003C00FCFF82FF7B00028822F480620A438B
:1013600002807047028922F400420A4302817047DA
:10137000028822F00A020A430280704770B586B0E4
:10138000044616460D46684600F08AFBA08802997E
:1013900020F03F022648B1FBF0F080B2202800D9AF
:1013A00020200243A280228822F001022280226AA9
:1013B00022F03F031F4A954212D86A00B1FBF2F1B6
:1013C00089B2042900D20421401C00F03F001843D8
:1013D0002062A183208840F00100208006B070BD0B
:1013E000B6F5804F05D005EB4502B1FBF2F18AB2AC
:1013F00008E005EBC50202EB0512B1FBF2F189B280
:1014000041F48042110501D142F001020A4E42F43A
:1014100000414FF47A72B54203D84FF49675684391
:1014200002E0C0EB0010C000B0FBF2F0CCE700001F
:1014300040420F00A0860100801A0600818941F019
:10144000010181817047C9438182704770B50C46A4
:10145000CA8805460968FFF791FFA1882846FFF76B
:1014600087FF61892846FFF777FFA1892846FFF7A4
:1014700079FF21892846BDE8704000F01EB841F28E
:1014800088310160002181804BF6FF72C2800181AA
:1014900041814FF480418181704782880A43828074
:1014A0007047818A008B41EA004121F07F407047FC
:1014B000018841F001010180704702896FF3090240
:1014C0000A4302817047828901F0FE0122F0FE0288
:1014D00011438181704700000449884202D14FF4D2
:1014E000001001E04FF4800000F0BEBA005400404C
:1014F00030B58BB04FF4807000F09EFA4FF480004E
:1015000000F0AAFA6846FFF7F4FB4FF44060009041
:10151000122001900720059000240120CDE902044B
:1015200069461748FFF7A6FB164D2846FFF7D4FF7C
:1015300006A8FFF7A4FF29144C20ADF820000811DD
:10154000ADF82200ADF81C400F48ADF81E10ADF804
:101550002410069046212846FFF7B5FF2846FFF7DE
:101560006DFF06A92846FFF771FF4FF4E06128469A
:10157000FFF793FF2846FFF79BFF0BB030BD00003D
:101580000038024000580040A086010030B500211C
:10159000034608464FF6FF74012505FA01F204EAF6
:1015A00040001A4201D040F00100491CC9B2102984
:1015B000F3D330BD02490843024908607047000078
:1015C0000000FA050CED00E010B54FF48004204651
:1015D00000F04AFA204600F037FA204600F044FABC
:1015E000FFF786FF202001F052FCBDE810402120CB
:1015F00001F04DBC38B5174C00200090144D206808
:1016000020F080002060206840F0400020606946A3
:101610001148A8470098C0B2052814D869460F4859
:10162000A84700984FF47F42010E02EA10221143AE
:1016300000F47F400A4A41EA00210091106800F05E
:101640007F4008431060206840F08000206038BD73
:10165000A502FF1F0020024020F0FF1F30F2FF1FF5
:101660000418004010B54FF480342046FFF746F8C8
:1016700000280AD005490120087005A001F0EAFB06
:101680002046BDE81040FFF733B810BD4E000020E3
:10169000700A00001CB54FF0805000F0DDF968467C
:1016A000FFF757F84FF480342046FFF721F8002069
:1016B0008DF8040010208DF8050001208DF806003B
:1016C00000946846FFF734F8E02000F009F803487A
:1016D000016841F0100101601CBD00000070004075
:1016E000034A116821F4387101431160704700000A
:1016F000007000402DE9FF4F494D00264FF6FF7165
:101700000D9C0123A982484F4649F960DFF820A1CA
:1017100046490AF1020BAE462AE030F816502F0A6D
:101720008EF8107010F816708EF8107030F8169051
:101730000F251AF80380B1F800C008FA04F829FA56
:1017400005F74CEA080C07F0010721F802CB0BEB78
:101750004303DB5D31F8027B03FA04FC6D1E47EAAC
:101760000C076DB221F8027C002DE2DA761CF6B28D
:10177000019DAE42D1D30025D9462AE032F81500AA
:10178000060A8EF8106012F815608EF8106032F8B4
:1017900015700F201AF80380B1F800C008FA04F899
:1017A00027FA00F64CEA080C06F0010621F802CBF5
:1017B00009EB43039B5D31F8026B03FA04FC401E06
:1017C00046EA0C0640B221F8026C0028E2DA6D1CF1
:1017D000EDB203988542D1D3BEF814500F2056467F
:1017E0005F4616F80380B1F800C008FA04F825FA3D
:1017F00000F24CEA080C02F0010221F802CB07EBE0
:1018000043039B5C31F8022B03FA04FC401E42EABE
:101810000C0240B221F8022C0028E2DABDE8FF8F6A
:101820000030024000340240F0090020C4160020BD
:10183000E10000202DE9F047DFF864900E464FF6F6
:10184000FF711D46904607460024A9F8141045F282
:10185000555018807200981C3946FEF777FC701CB2
:1018600080B24B4608E037F81410090A197417F8CB
:1018700014101974641CA4B2B442F4D3002108E01B
:1018800035F81020140A1C741A74401C491C80B2CC
:1018900089B24145F4D3998A25F81010BDE8F08744
:1018A0000030024070B5324C00203021A073A1817D
:1018B0000C21E17349F6EF51A18244F2FF31E1803E
:1018C0004FF4004121810621A1722A4921612A4950
:1018D00021622A49054600EBC002C2EB801204EBEC
:1018E000800301EB42025A63401CE27BC0B2824299
:1018F000F1D8102060701C20207001016180C81C8C
:10190000A0801FA001F0A6FA217822A001F0A2FA7F
:10191000617825A001F09EFA607F08B127A100E060
:101920002AA12EA001F096FAE17B30A001F092FAF4
:10193000A27AA18933A001F08DFA47F2305060837A
:101940004FF4967020833B4840F2F521C1803D2141
:101950000181E188418122890282418482848562F9
:1019600080F821500221C17501210177457070BDB9
:10197000140A00200C000020DC3400087C0A00203F
:1019800070726F6A656374207A6F6E65733A25644E
:101990000A00000070726F6A65637420776964746E
:1019A000683A25640A00000070726F6A65637420EB
:1019B0006865696768743A25640A00006869676841
:1019C000207370656564206D6F6465006C6F7720AF
:1019D0007370656564206D6F6465000073706220CC
:1019E0006D6F64653A25730A0000000070726F6ABB
:1019F000656374206469206E756D626572733A2543
:101A000064200A0070726F6A6563742064692063E1
:101A10006173636164653A2564202C206963206EDC
:101A2000756D62657220706572206469703A256414
:101A30000A0000001C06002002494A6902434A616C
:101A400070470000001002400249CA698243CA611F
:101A500070470000001002400249CA690243CA618F
:101A6000704700000010024003490A6902430A61FE
:101A70000A6982430A6170470010024002498A697C
:101A800002438A6170470000001002400349CA689F
:101A90000243CA60CA688243CA60704700100240AD
:101AA00030B5284B5968284A11405A680C0102F495
:101AB000803201D4022401E06FF4F77404EB914109
:101AC0001AB15A68920305D502E01A6CD20701D008
:101AD0001E4A00E01E4A51435A681D4C12F00C0287
:101AE00003D0042A01D0082A01D0046000E001607C
:101AF0005A68184CC2F30312A55C0268EA404260BF
:101B00005D68C5F30225655D22FA05F585605D68AF
:101B1000C5F3C225645D22FA04F4C460DC6A0D4D8D
:101B200004F00F0410352C5DB2FBF4F24261DA6A66
:101B300005F11003C2F3031233F81220B1FBF2F1E6
:101B4000016130BD0010024000003C0800093D006A
:101B500000127A006C3C0008028822F038020280F1
:101B600002880A4302807047028822F00102028044
:101B700002880A4302807047028822F00202028033
:101B800002880A4302807047028822F4444202809D
:101B900002880A4302807047028822F400620280B1
:101BA00002880A4302807047028822F08002028085
:101BB00002880A430280704782880A438280704705
:101BC0000649884201D1801404E00549884203D1C6
:101BD0004FF40020FFF75ABF70470000003001406B
:101BE000003C014010B50B4604460988FFF7CCFFC6
:101BF0005988204600F034F899882046FFF7CCFF3A
:101C000019892046FFF7B0FFD9882046FFF7B4FFB7
:101C10005989204600F017F899892046FFF79CFF64
:101C2000D9892046FFF7C0FF188A208210BD002105
:101C3000018041808180C180018141818181C18198
:101C4000072101827047028822F400720280028814
:101C50000A4302807047018821F0400101807047EB
:101C6000028822F00402028002880A430280704740
:101C700010B54FF4A060FFF79DFC0120FFF7FEFEBA
:101C800000211B2001F010F900211C2001F00CF9AB
:101C90000521162001F008F905210B2001F004F9B7
:101CA0000A210D2001F000F909211D2001F0FCF8A6
:101CB0000921202001F0F8F80A21212001F0F4F890
:101CC00009211D2001F0F0F80A212F2001F0ECF885
:101CD0000F21012001F0E8F80A21302001F0E4F89A
:101CE0000A21242001F0E0F80121062001F0DCF8AF
:101CF0000121072001F0D8F80121082001F0D4F8D3
:101D00000121092001F0D0F801210A2001F0CCF8CE
:101D10000121272001F0C8F81B2001F0ABF81C209E
:101D200001F0A8F8272001F0A5F8062001F0A2F89C
:101D3000072001F09FF8082001F09CF8092001F02D
:101D400099F80A2001F096F80B2001F093F80D2085
:101D500001F090F81D2001F08DF82F2001F08AF895
:101D6000012001F087F8162001F084F8202001F00E
:101D700081F8212001F07EF8302001F07BF824204A
:101D800001F078F8BDE81040802000F0E1BC0000D0
:101D90001549CA6842F40022CA60CA6822F40022C7
:101DA000CA608A6942F400228A61104900230B80CC
:101DB0000A1D1380138843F0010313800A8842F43C
:101DC00020620A800A8842F040020A8008498A6834
:101DD00022F001028A60074A4A61C860886840F0C0
:101DE000010088607047000000100240003C014084
:101DF000000002405806002070B5324D90B02846D1
:101E0000FFF7DEFE4FF40020FFF738FE0120FFF75A
:101E100013FE0BA8FFF70BFF0024E814ADF8300009
:101E2000ADF834408010ADF836000120ADF82C40FC
:101E3000ADF83840ADF83C00ADF82E40ADF832407A
:101E4000ADF83A400BA92846FFF7CCFE1E4E3046AF
:101E5000FEF722FB6846FEF76DFB1A4869460C3018
:101E600000901A48C068CDE901041020CDE90304B0
:101E700080200590400006908000CDE907044FF4D3
:101E80004050CDE909043046FEF7ABFA0E49083957
:101E90004C60886840F002008860886940F00B0060
:101EA000886101212846FFF787FE0C213046FEF7A6
:101EB00086FA3046FEF77EFA2846FFF7CCFE10B0D1
:101EC00070BD0000003C014008000240E009002015
:101ED00010B586B08020FFF7AFFD6846FEF709FF1A
:101EE00001200021274C0190039100906946204673
:101EF000FEF7C0FE0221009169462046FEF7BAFEB9
:101F00000421009169462046FEF7B4FE08210091A5
:101F100069462046FEF7AEFE202000906946204626
:101F2000FEF7A8FE4020009069462046FEF7A2FE7C
:101F30008020009069462046FEF79CFEA015009088
:101F400069462046FEF796FE201500906946204619
:101F5000FEF790FEE014009069462046FEF78AFEE8
:101F6000A014009069462046FEF784FE4FF400401E
:101F7000009069462046FEF77DFEFEF70DFB06B099
:101F800010BD00000034024030B50D4801780D4A04
:101F9000002341B114880C4908888D680544401C11
:101FA00008802C700AE00121017006481438036093
:101FB00004482438016841F001010160138030BDFC
:101FC000E000002024080040040A002070B54FF40F
:101FD00080758AB02846FFF72FFDA800FFF72CFD7B
:101FE0000120FFF74BFD0420FFF736FD0820FFF727
:101FF00033FD6846FEF77DFE00240121CDE9021481
:10200000684E0091019469463046FEF733FE012187
:102010000020FEF7FBFD0220009069463046FEF7E7
:1020200029FE05210120FEF7F1FD042000906946FC
:102030003046FEF71FFE09210220FEF7E7FD0820CB
:10204000009069463046FEF715FE0D210320FEF78D
:10205000DDFD1020009069463046FEF70BFE112191
:102060000420FEF7D3FD2020009069463046FEF79D
:1020700001FE15210520FEF7C9FD402000906946AC
:102080003046FEF7F7FD19210620FEF7BFFD802040
:10209000009069463046FEF7EDFD1D210720FEF752
:1020A000B5FD694630460095FEF7E4FD2121082084
:1020B000FEF7ACFD6800009069463046FEF7DAFD99
:1020C00025210920FEF7A2FDA801009069463046AF
:1020D000FEF7D0FD39210E20FEF798FDE8010090B3
:1020E00069463148FEF7C6FD3F210F20FEF78EFD01
:1020F0002E49C888098908432D490A6882430A6025
:102100002B4908310A6802430A60091D0A68104316
:10211000086006A800F066FC9F20ADF81C000325AF
:10212000244EADF81850ADF81E40ADF81A4006A97F
:10213000304600F0FDFB304600F0C6FB2946304635
:1021400000F04EFC1B491031086820F001000860C7
:102150000121304600F07BFC06A800F043FC40F66D
:102160009F70ADF81C00ADF81840ADF81E40ADF8FA
:102170001A40114C0F2506A9204600F0D9FB204635
:1021800000F0A2FB2946204600F02AFC0A49103143
:10219000086820F0010008600121204600F057FC8B
:1021A0000AB070BD0038024000400240140A00200E
:1021B0000004014000080040000C004010B5FFF78B
:1021C00087FEBDE81040FFF701BF00000548016829
:1021D00021F0010101600448016821F00101016062
:1021E0007047000000080040000C00407FB501204F
:1021F000FFF732FC0220FFF72FFC684600F0F2FBED
:1022000005200024ADF80400ADF80040850706263F
:10221000ADF80640ADF802406946284600F088FB5C
:10222000284600F051FB3146284600F0D9FB2869CA
:1022300020F0010028610121284600F008FC6846D2
:1022400000F0D0FB0420ADF80400ADF80040ADF87C
:102250000640ADF802400C4C08256946204600F0C7
:1022600067FB204600F030FB2946204600F0B8FB13
:1022700005491031086820F001000860012120465E
:1022800000F0E5FB7FBD00000004004038B50022EF
:10229000ADF800200C4A47F2B04340EA012412781E
:1022A00043EA0215094A137C002BFCD10848807BC5
:1022B00000B1012001F0E4F86B46002221462846D7
:1022C00000F092F838BD000084180020F0090020CA
:1022D000140A0020F7B5094B0446002542F4E446F1
:1022E000187C0028FCD1012001F0CAF801AB22467D
:1022F0002946304600F078F8FEBD0000F0090020C5
:10230000F0B41B0205460A48A3F580730B43120282
:102310000078A2F58072049C4FF4E64699B22A43F5
:1023200046EA00102346F0BC92B200F0C5B80000A7
:1023300084180020F0B414460646DDE90425094857
:102340000170807840EA01104FF4E24141EA460111
:1023500008431902A1F5807121432B46F0BC89B2D4
:1023600000F0AAB88418002010B5FFF727FFFFF788
:102370003DFF4020FFF760FBBDE81040012001F069
:102380007FB8002245F6C3217820FFF7A3BF0000E5
:10239000F8B504460020ADF8000010484FF4EA45B7
:1023A000007845EA00161802A0F58070084385B24F
:1023B0001002A0F580702043094B84B2187C0028DD
:1023C000FCD10848807B00B1012001F059F86B4630
:1023D00022462946304600F007F8F8BD8418002050
:1023E000F0090020140A00202DE9FF410F460146A4
:1023F000002001900290039098461446ADF8041016
:102400003846FFF7C3F8ADF806002046FFF7BEF8E0
:10241000ADF808001F480189ADF80A104089FFF7A0
:10242000B5F8ADF80C0005264FF4E0711A48FDF739
:10243000A6FE0824194D0AE0286901234246005DE2
:102440000090314601A8FFF755F9641CE4B2E87B1F
:10245000A042F1D86FF0010000EB172060F31F27B6
:10246000B8B2FFF793F8ADF80600002428690123FD
:102470004246005D0090314601A8FFF73BF9641C1D
:10248000E4B2082CF2D34FF480700121FEF790F8EB
:10249000BDE8FF8184180020C4160020140A002023
:1024A00000224AF2C9517820FFF714BF00224AF2F5
:1024B000C9517C20FFF70EBF2DE9FE430024009494
:1024C000ADF800001D461646019402940846FFF739
:1024D0005DF8ADF802003046FFF758F8ADF804009B
:1024E00016480189ADF806104089691E084380B27C
:1024F000FFF74CF8ADF80800280170304FF00509DF
:102500001FFA80F80E4E0F4F0CE004EBC400C0EB36
:10251000841006EB40032A4649466846FFF78AF9CD
:10252000641CE4B2F87BA042EFD84046FDF796FE6B
:1025300001214046FEF70CF8BDE8FE838418002018
:102540007C0A0020140A00200648016811B10168C5
:10255000491E01608168002902D04168491C416020
:10256000704700001800002070B586B00120FFF70A
:1025700085FA4FF48070FFF75FFA6846FEF7B9FB03
:1025800001244FF4005002250594CDE900050D4EBD
:1025900069463046FEF76EFB20030594CDE9000541
:1025A00069463046FEF766FBE0030090002001908C
:1025B000694605943046FEF75DFB06B0BDE8704005
:1025C000FFF71ABC003802403EB5002000908DF89D
:1025D0000400324C0290206840F0010020604FF46B
:1025E000A0612068C0F340008DF804000298401CF0
:1025F00002909DF8040010B902988842F1D1206839
:10260000C0F340008DF804009DF80400F0B32448A6
:10261000016821F00701016022490968016841F061
:102620000301016060686060606840F400506060B1
:10263000606840F4A0606060FEF7DCFF60681A49E3
:1026400008406060206C20F0010020646068019008
:102650000098164940F0010000900198084301904D
:10266000606000982064206840F0807020602068DE
:102670008001FCD5606820F003006060606840F075
:10268000020060606068C0F3810000E002E00228A0
:10269000F8D13EBD0749064808603EBD0010024023
:1026A00000200240002004E0FFFFC0F700003C08CB
:1026B00000127A000C0100201E4810B5016841F498
:1026C000700101601C48016841F00101016041682E
:1026D0001A4A114041600168194A114001600168BD
:1026E00021F4802101604168164A114041604FF495
:1026F0006051C162016C41F00101016412498160C5
:10270000C16941F08051C161C16921F08051C1614D
:102710000E48016841F080010160016821F010015C
:102720000160FFF751FF03494FF0006080390860F6
:1027300010BD000088ED00E0001002400CC07FF8E2
:10274000FFFFF6FEFFFFC0F700009F0400200240DD
:102750004FF47A7148434FF0E02100220A6148614A
:102760008A6106200861704770B5104C20681049D6
:10277000898A4840231D1860002519070D610D48FE
:102780000288521C028002884688B24204D10A683C
:1027900022F001020A600D612168826812885140AE
:1027A00019608168891C816070BD0000103402408E
:1027B000140A0020F0090020104810B50021016023
:1027C0000F48028843889A4209D28168028831F80A
:1027D0001210C26851610188491C018010BD094B6B
:1027E0001A68094CA48A22431A60044A103A1368F2
:1027F00023F001031360017410BD000010040040B9
:10280000F009002014340240140A00200E4A00B5DA
:102810001068C00717D0FFF7D9FC106820F001003E
:10282000106009490020143108800848C1880089D7
:102830000143074802688A43026004481038017B5C
:1028400041F00101017300BD10080040140A00208E
:10285000000401400E4800B5016821F0010101604B
:102860000C4A5068401E5060506800280ED1FFF797
:10287000ADFC08481030C188008901430648036850
:102880008B430360107B40F00200107300BD00001A
:10289000100C0040040A00200004014008480169AF
:1028A00021F00101016107480188491C018001886C
:1028B000B1F5FA6F02D34FF4C86101807047000090
:1028C000001000404C000020016841F080010160D0
:1028D00070470029016802D041F4006101E021F451
:1028E0000061016070470029016802D041F4805105
:1028F00001E021F48051016070470029016802D095
:1029000041F4005101E021F40051016070470029B9
:10291000016802D041F4804101E021F4804101606E
:102920007047026822F070020A430260704700009C
:1029300070B5214D0C460346A84206D06188FFF7CA
:10294000F0FFE188184600F074F8A0889885208888
:1029500018851A4A1A4E934201D0B34201D1207A07
:10296000188601209882AB4203D0617A1846FFF79F
:10297000B0FF4FF08045934209D0B34207D0AB423D
:1029800005D01048834202D00F48834213D1617BA7
:10299000184600F01BF8AB420DD1A17A1846FFF79C
:1029A000A2FFE17A1846FFF7A8FF217BBDE870403F
:1029B0001846FFF7ACBF70BD00100040002C01406E
:1029C0000034014000040040000800400029016874
:1029D00002D041F4004101E021F400410160704760
:1029E000018570474FF6FF71818000210180C18011
:1029F0004180017241728172C172017341738173AE
:102A00007047026A01238B409A4302627047026A50
:102A100001238B401A4302627047026A04238B40F1
:102A20009A4302627047026A04238B401A4302628F
:102A30007047026822F44072026002680A43026032
:102A40007047C26B6FF30F020A43C26370478289FB
:102A50000A4382817047C94301617047016821F0D0
:102A6000010101607047016841F001010160704798
:102A7000F0B50C4605460821FFF7C3FF6E68E8690C
:102A8000278880B220F07300074321890822284656
:102A900000F03BF860884FF008010028284602D07B
:102AA000FFF7B5FF01E0FFF7ACFF1148854202D008
:102AB0001048854217D161890822284600F01CF889
:102AC000A0884FF008010028284602D0FFF7ABFF8E
:102AD00001E0FFF7A2FFA18926F4405040EA01106F
:102AE000E18940EA01166E60EF61E088E863F0BDBD
:102AF000002C01400034014010B5036A08249440C2
:102B0000A34391401943016210BD10B5036A02242A
:102B10009440A34391401943016210BD30F8441F13
:102B200041F40041018070472DE9FC412F494FF0ED
:102B30000108002481F801802B4D4FF4A5612C4839
:102B4000FDF71DFBDFF8A8C040F6FF720020C4EBC4
:102B5000C40700EB8701401C35F8111080B201F06A
:102B60000F03C1F3061603EBC603C90A01EBC10646
:102B7000C6EB81110CEB410101EB43011C288A815A
:102B8000E7D3641CA4B2102CE0D31A4C00253020EB
:102B900084F802806581CDE900501748012246463D
:102BA000837A11462846FFF7C5FBC82000F0E5FBF5
:102BB0004FF480406081182240F299117A20FFF78B
:102BC00089FBC82000F0D9FB0123267065811A46D5
:102BD00019461320FFF7DCFBC82000F0CEFBBDE850
:102BE000FC41052000F0B1BBDC34000800000020EF
:102BF0007C0A002084180020140A002030B587B019
:102C000004460D466846FEF74BFF1448844205D043
:102C100013498C4202D013498C4201D1039A00E03F
:102C2000029AA90002EBC20000EB0210B0FBF1F126
:102C30006423B1FBF3F0020110096FF0180568433B
:102C400001EB8000322101EB0010B0FBF3F000F04B
:102C50000F001043208107B030BD00000038014054
:102C60000050014000540140C1F3080181807047C9
:102C7000818941F40051818170470088084000D06B
:102C800001207047828A22F440720A438282704790
:102C900070B50C4605460968FFF7B0FFA1882846C5
:102CA00000F053F8E188284600F03EF821892846D4
:102CB00000F010F86189284600F006F8A18928463E
:102CC000BDE87040FFF7DEBF828922F00C020A43A4
:102CD00082817047828922F4C0620A4382817047F0
:102CE0000D49884202D14FF4804011E00B494FF466
:102CF0000032884202D11046FEF7B6BE084988422B
:102D000001D1104604E00749884203D14FF48020E6
:102D1000FEF7BCBE70470000003801400044004090
:102D20000050014000540140028A22F440520A43FC
:102D3000028270474FF41651016000218180C180EA
:102D400001810C22428181817047828922F4805264
:102D50000A4382817047000030B504468BB04FF4BF
:102D60008070FEF769FE44F20100FEF787FE04A8BA
:102D7000FDF7BFFF4FF4007004900220059005207E
:102D8000099004A90F48FDF775FF0F4D2846FFF77E
:102D9000A7FF6846FFF7CEFF0020ADF80400ADF8AE
:102DA0000600ADF80800ADF80C000820ADF80A00E8
:102DB000009469462846FFF76BFF2846FFF758FF47
:102DC0000BB030BD00340240003801401CB500F0AB
:102DD00019F80120FEF752FE36210D20FDF716FFEF
:102DE0004FF40050009000208DF8040008208DF86A
:102DF000050001208DF806006846FDF799FC00F0FB
:102E000021F81CBD00B587B04FF40070FEF714FE2A
:102E10006846FDF76EFF00200221CDE90101039015
:102E20000803009069460248FDF724FF07B000BD83
:102E3000003C02400248016841F4005101607047C3
:102E4000080401400248016821F400510160704704
:102E5000080401400FB4054B10B503A9044A0298B9
:102E600000F042F810BC5DF814FB0000A533000828
:102E700010010020002809DB00F01F020121914011
:102E80004009800000F1E020C0F8001170470028E0
:102E900009DB00F01F02012191404009800000F190
:102EA000E020C0F8001170470907090E002804DB74
:102EB00000F1E02080F80014704700F00F0000F1EE
:102EC000E02080F8141D704702E008C8121F08C1F6
:102ED000002AFAD170477047002001E001C1121F9B
:102EE000002AFBD1704700002DE9FF4F8DB00F463F
:102EF0000546002606E025280BD0DDE90F12904795
:102F00006D1C761C28780028F5D111B03046BDE83C
:102F1000F08F0024A246A1460122EC4900E00443C0
:102F200015F8013F203B02FA03F00842F7D1287858
:102F30002A2810D06FF02F022878A0F1300109293B
:102F400014D80AEB8A0102EB410144F0020400EBC1
:102F5000010A6D1CF0E701CF5FEA000A03D544F4D3
:102F60000054CAF1000A44F002046D1C28782E288F
:102F700017D115F8010F44F004042A280ED06FF081
:102F80002F022878A0F1300109290AD809EB89011C
:102F900002EB410100EB01096D1CF2E757F8049BBD
:102FA0006D1C28786C280FD006DC4C2817D06828B8
:102FB0000DD06A2814D104E0742810D07A280FD1DB
:102FC0000DE044F400140AE044F4801401E044F4F9
:102FD00040146978814202D104F580146D1C6D1C87
:102FE0002A786E2A1FD00CDC632A31D004DC002A38
:102FF0008BD0582A11D1A3E0642A68D0692A0CD159
:1030000065E0732A2ED004DC6F2A73D0702A04D1B5
:103010009BE0752A6FD0782A6ED01046DDE90F123A
:103020009047761C50E1C4F30250022806D00328D2
:1030300009D0042801CF09D0066045E101CFF1177E
:10304000C0E9006140E101CF06803DE106703BE14F
:1030500017F8040B8DF8000000208DF80100EB46F6
:10306000012003E057F804BB4FF0FF3061074FF039
:10307000000102D40DE008F10101884649450FDA4C
:103080008045F8DB1BF808100029F4D108E008F1AE
:10309000010188468142FADB1BF808100029F6D1AD
:1030A000DDE90F23AAEB08008146214600F036F93E
:1030B000304400EB080604E0DDE90F121BF8010BB9
:1030C0009047B8F10108F7D221464846F7E00A21B7
:1030D000C4F302534FF0000B0891022B04D001CF30
:1030E000C117032B09D00AE0FF1D27F00707F7E8F7
:1030F000020108E032E01FE020E000B2C117042B1B
:1031000001D140B2C117031E71F1000307DA4FF07D
:10311000000CD0EB0C006CEB01012D2302E0230529
:1031200004D52B238DF82430012303E0E30701D0DD
:103130002023F7E7984658E00A2110E010210EE01E
:1031400010204FF0000B08900CE010214FF0000B06
:1031500044F004044FF00809089103E008214FF0FF
:10316000000B0891C4F30253022B04D001CF0021BD
:10317000032B06D006E0FF1D27F00707F7E8020142
:1031800003E080B2042B00D1C0B24FF00008230747
:103190002BD5702A07D0DDF820C08CF0100C5CEA2B
:1031A0000B0C05D00EE040238DF82430012308E0FD
:1031B00050EA010306D030238DF824308DF8252005
:1031C00002239846DDF820C08CF0080C5CEA0B0C5A
:1031D0000BD150EA010301D1630706D530238DF8E6
:1031E00024304FF00108A9F10109582A04D038A26F
:1031F0000B9208AA0A920BE03AA2F9E75B46089AFA
:10320000FCF7C8FF0B9B9B5C0A9A521E0A92137034
:1032100050EA0102F2D10A98ADEB000000F1200B58
:10322000600702D524F4803401E04FF00109D9454C
:1032300002DDA9EB0B0000E0002000EB0B01414494
:103240000890AAEB010AE00306D4DDE90F2321462A
:10325000504600F063F806444FF0000908E009A961
:1032600011F80900DDE90F12904709F10109761CF8
:10327000C145F4DBE0030CD5DDE90F2321465046C0
:1032800000F04CF8064404E0DDE90F1230209047CE
:10329000761C0899481E08900029F5DC08E00A9879
:1032A0000A990078491C0A91DDE90F129047761CB3
:1032B000BBF10001ABF1010BF1DC21465046DDE929
:1032C0000F2300F019F806446D1C1BE609280100C5
:1032D000303132333435363738396162636465668C
:1032E000000000003031323334353637383941424E
:1032F00043444546000000002DE9F0410446002506
:103300001E461746880404D405E039462020B047FD
:103310006D1C641EF9D52846BDE8F0812DE9F04109
:10332000044600251E469046C80301D5302700E01C
:103330002027880404D505E041463846B0476D1C77
:10334000641EF9D52846BDE8F081822800D9822084
:103350004FF0E02104230B614FF4FA3250434861EF
:1033600000228A61052008610869000CFCD00B610D
:103370004FF4FA3048618A6170474FF0E02104222F
:103380000A61C001486100238B610520086108695A
:1033900010F4803FFBD00A614FF4FA3048618B6132
:1033A0007047000070B50D4D04460A2809D10D2163
:1033B0002846FFF759FC80212846FFF75EFC0028CD
:1033C000F9D0E1B22846FFF74FFC80212846FFF7ED
:1033D00054FC0028F9D0204670BD000000380140A0
:1033E000FEF746FC4FF46120FFF7B6FCFEF75AFAF1
:1033F000FEF750F91C48018B408BFDF761FBFEF78F
:10340000B3FFFCF77FFF19A0FFF724FD002240F671
:10341000FF714220FDF7A4FDFEF76AF8FFF7A4F85C
:10342000FFF7D4FC4FF4FA70FDF720FBFDF710FB1B
:10343000FFF700FD3D20FDF705FB104CFFF774FB87
:10344000C820FFF79AFFE07D28B9A07E18B1207F41
:1034500008B1FDF7B1F9102200212F20FEF73AFF45
:10346000FDF77EFAEAE70000140A00207374617227
:103470007420696E69742069630A00001C060020CC
:1034800010B50B480021094C828A0B4604EB011051
:10349000491C038043808280C380028142818381F2
:1034A000C9B2C2810429F1D310BD000084160020E6
:1034B000140A002010B5034C2070A180E280238103
:1034C00010BD00008418002010B5034C20706170FE
:1034D000A270638110BD000084180020300810081D
:1034E000300010003018101830101010302810283C
:1034F000302010203038103830301030304810482C
:1035000030401040305810583050105050585050E3
:10351000504850403108110831001100311811187D
:103520003110111031281128312011203138113873
:103530003130113031481148314011403158115863
:1035400031501150515851505148514032081208D1
:1035500032001200321812183210121032281228BB
:1035600032201220323812383230123032481248AB
:103570003240124032581258325012505258525063
:1035800052485240330813083300130033181318FD
:1035900033101310332813283320132033381338F3
:1035A00033301330334813483340134033581358E3
:1035B0003350135053585350534853403408140851
:1035C000340014003418141834101410342814283B
:1035D000342014203438143834301430344814482B
:1035E00034401440345814583450145054585450E3
:1035F000544854403508150835001500351815187D
:103600003510151035281528352015203538153872
:103610003530153035481548354015403558155862
:1036200035501550555855505548554036081608D0
:1036300036001600361816183610161036281628BA
:1036400036201620363816383630163036481648AA
:103650003640164036581658365016505658565062
:1036600056485640370817083700170037181718FC
:1036700037101710372817283720172037381738F2
:1036800037301730374817483740174037581758E2
:103690003750175057585750574857402008000880
:1036A00020000000201800182010001020280028FA
:1036B00020200020203800382030003020480048EA
:1036C00020400040205800582050005040584050A2
:1036D000404840402108010821000100211801183C
:1036E0002110011021280128212001202138013832
:1036F0002130013021480148214001402158015822
:10370000215001504158415041484140220802088F
:103710002200020022180218221002102228022879
:103720002220022022380238223002302248024869
:103730002240024022580258225002504258425021
:1037400042484240230803082300030023180318BB
:1037500023100310232803282320032023380338B1
:1037600023300330234803482340034023580358A1
:10377000235003504358435043484340240804080F
:1037800024000400241804182410041024280428F9
:1037900024200420243804382430043024480448E9
:1037A00024400440245804582450045044584450A1
:1037B000444844402508050825000500251805183B
:1037C0002510051025280528252005202538053831
:1037D0002530053025480548254005402558055821
:1037E000255005504558455045484540260806088F
:1037F0002600060026180618261006102628062879
:103800002620062026380638263006302648064868
:103810002640064026580658265006504658465020
:1038200046484640270807082700070027180718BA
:1038300027100710272807282720072027380738B0
:1038400027300730274807482740074027580758A0
:103850002750075047584750474847404D43555613
:103860006572040504055F011C10200000000000C3
:10387000B71DC1046E3B8209D926430DDC760413C3
:103880006B6BC517B24D861A0550471EB8ED08265A
:103890000FF0C922D6D68A2F61CB4B2B649B0C35F7
:1038A000D386CD310AA08E3CBDBD4F3870DB114CA4
:1038B000C7C6D0481EE09345A9FD5241ACAD155F87
:1038C0001BB0D45BC2969756758B5652C836196A90
:1038D0007F2BD86EA60D9B6311105A6714401D797B
:1038E000A35DDC7D7A7B9F70CD665E74E0B6239825
:1038F00057ABE29C8E8DA191399060953CC0278B8F
:103900008BDDE68F52FBA582E5E66486585B2BBE15
:10391000EF46EABA3660A9B7817D68B3842D2FAD32
:103920003330EEA9EA16ADA45D0B6CA0906D32D4D5
:103930002770F3D0FE56B0DD494B71D94C1B36C70A
:10394000FB06F7C32220B4CE953D75CA28803AF213
:103950009F9DFBF646BBB8FBF1A679FFF4F63EE16E
:1039600043EBFFE59ACDBCE82DD07DEC7770863433
:10397000C06D4730194B043DAE56C539AB068227A2
:103980001C1B4323C53D002E7220C12ACF9D8E12E1
:1039900078804F16A1A60C1B16BBCD1F13EB8A0116
:1039A000A4F64B057DD00808CACDC90C07AB9778A3
:1039B000B0B6567C69901571DE8DD475DBDD936BE6
:1039C0006CC0526FB5E6116202FBD066BF469F5EC7
:1039D000085B5E5AD17D1D576660DC5363309B4D9A
:1039E000D42D5A490D0B1944BA16D84097C6A5AC28
:1039F00020DB64A8F9FD27A54EE0E6A14BB0A1BFEE
:103A0000FCAD60BB258B23B69296E2B22F2BAD8A1C
:103A100098366C8E41102F83F60DEE87F35DA999D1
:103A20004440689D9D662B902A7BEA94E71DB4E094
:103A3000500075E4892636E93E3BF7ED3B6BB0F369
:103A40008C7671F7555032FAE24DF3FE5FF0BCC64A
:103A5000E8ED7DC231CB3ECF86D6FFCB8386B8D58D
:103A6000349B79D1EDBD3ADC5AA0FBD8EEE00C696D
:103A700059FDCD6D80DB8E6037C64F643296087A73
:103A8000858BC97E5CAD8A73EBB04B77560D044FC6
:103A9000E110C54B383686468F2B47428A7B005C47
:103AA0003D66C158E4408255535D43519E3B1D2500
:103AB0002926DC21F0009F2C471D5E28424D193637
:103AC000F550D8322C769B3F9B6B5A3B26D615037C
:103AD00091CBD40748ED970AFFF0560EFAA01110CB
:103AE0004DBDD014949B93192386521D0E562FF171
:103AF000B94BEEF5606DADF8D7706CFCD2202BE2BF
:103B0000653DEAE6BC1BA9EB0B0668EFB6BB27D701
:103B100001A6E6D3D880A5DE6F9D64DA6ACD23C402
:103B2000DDD0E2C004F6A1CDB3EB60C97E8D3EBD11
:103B3000C990FFB910B6BCB4A7AB7DB0A2FB3AAE3A
:103B400015E6FBAACCC0B8A77BDD79A3C660369B7F
:103B5000717DF79FA85BB4921F4675961A1632883E
:103B6000AD0BF38C742DB081C330718599908A5D53
:103B70002E8D4B59F7AB085440B6C95045E68E4ED2
:103B8000F2FB4F4A2BDD0C479CC0CD43217D827B4D
:103B90009660437F4F460072F85BC176FD0B8668E6
:103BA0004A16476C93300461242DC565E94B9B117F
:103BB0005E565A1587701918306DD81C353D9F0216
:103BC00082205E065B061D0BEC1BDC0F51A69337B3
:103BD000E6BB52333F9D113E8880D03A8DD097246A
:103BE0003ACD5620E3EB152D54F6D4297926A9C5F4
:103BF000CE3B68C1171D2BCCA000EAC8A550ADD69E
:103C0000124D6CD2CB6B2FDF7C76EEDBC1CBA1E308
:103C100076D660E7AFF023EA18EDE2EE1DBDA5F021
:103C2000AAA064F4738627F9C49BE6FD09FDB88950
:103C3000BEE0798D67C63A80D0DBFB84D58BBC9A19
:103C400062967D9EBBB03E930CADFF97B110B0AFB6
:103C5000060D71ABDF2B32A66836F3A26D66B4BCDD
:103C6000DA7B75B8035D36B5B440F7B100000000EB
:103C70000102030401020304060708090102040605
:103C8000080A0C1020202020202020200100020003
:103C90000400060008000A000C001000200040008C
:103CA000800000010001000100010001CC3C00087F
:103CB0000000002014010000C82E0008E03D0008AC
:103CC000140100207C1B0000D82E00080001000019
:103CD00000000000000000000001020305060708C4
:103CE0000A0B0C0F000000000000000000000000A4
:103CF00000001100000FFF000000000000000000A5
:103D000000000000000000000000000000000000B3
:103D1000000000000000000000000000FF00FF00A5
:103D2000FF00FF0000000000FF00FF00FF00FF0099
:103D300000000000FF00FF00FF00FF000000000087
:103D4000FF00FF00FF00FF0000000000FF00FF0079
:103D5000FF00FF0000000000FF00FF00FF00FF0069
:103D600000000000FF00FF00FF00FF000000000057
:103D7000FF00FF00FF00FF0000000000FF00FF0049
:103D8000FF00FF00FF00FF00FF00FF00FF00FF003B
:103D9000FF00FF00FF00FF00FF00FF00FF00FF002B
:103DA000FF00FF00FF00FF00FF00FF000001000117
:103DB0000000010000000A0014001E00280032006C
:103DC0003C00460050005A0064006E0078008200FB
:103DD0008C009600A00000000020A1070000000059
:0400000508000115D9
:00000001FF
